:020000040000FA
:06000000FE300F306A28FB
:08000800A000030EA100831209
:10001000C31D3B288B1C34288B1031181628B11CAB
:10002000342864300102031833281A2800001828E5
:1000300019281A281B281C281D281E281F2820289C
:1000400021283110B114A810031005190314AA0DAA
:10005000A90DA80DB00B342831152A08AF002908C6
:10006000AE002808AD00B11081010B11210E8300F4
:10007000A00E200E090005194328831601178312CC
:10008000B23081005E2883160113831203140B190A
:100090000310A80DA90DAA0DAB0DAC0DAC16FF30C9
:1000A0002C02031D5E28FA302B02031D5E28311539
:1000B0002A08AF002908AE002808AD008B100B11EC
:0A00C000210E8300A00E200E09009F
:0C00D400203084008001840A8030040287
:1000E000031C6C281230B0005A30C000C10001302F
:1000F000D400D500E400E500E300F100F000EE00DC
:100100000730D8008030D7001F30E6000717FA30DC
:10011000FD000330EF008B13903003178D00831622
:100120008C130C1483120C080313C7008B1783164F
:100130000F308505203086050D3087058312850137
:1001400086018701103083168E008312703083166B
:100150008F00831200300317990003130030031738
:100160009A0003130030970000309F000030831680
:100170009F008312003003179E0003130030031703
:100180009F000313C030831681008312313090002A
:1001900000309200003083169400831200309400E7
:1001A000A630831698008312003083169B008312BA
:1001B00090309800333083169900831200308316F4
:1001C0008C008312003083168D00831210308B0058
:1001D0000D16DE2581018E018F010B118B100B1086
:1001E0008C128C018D010D168B172E2379238821FB
:1001F000E6170230C800332131192F24311A4D215E
:10020000591C11235918A2228F080319FB288F01AA
:10021000E422AF231922EB219F21C5211629E71BD8
:10022000EB01EB0B1629E801E901EA01E713591884
:10023000FB28B1192829D60BFB28B11A0A30B11EA8
:10024000C830D600B11A2F298821CC0ACC194A14FB
:10025000B111B11A0A30B11EC830D600FB2888216E
:10026000BE18DE25FB286400C31DB113C31D0800A2
:10027000311808000B1D08000B11B1103114123099
:10028000B000051D4829B117831601138312080019
:10029000B113831601178312080031124A10CC01E2
:1002A00021305B02031D5A295C08CE005D08CF0097
:1002B000661783295B085C065D02031D0800773022
:1002C0005B02031D67295C087406C400832966303D
:1002D0005B02031D6E295C08CB00832955305B024D
:1002E000031D75295C08F800832944305B02031D57
:1002F0007C295C08FA00832933305B02031D8329C3
:100300005C08FB008329B116B1110A30D600080041
:10031000591459158B138316071283128B1707165E
:1003200008005910D9101930DE00B112B111C830CF
:10033000D6008B138316071683128B170800051837
:10034000A6291930C0070318AB2908000A30C002DB
:10035000031CBD290800FF30C00042146430410274
:10036000031808004210C2144317C314F51BC3102E
:100370007717E6172830C8000800C0014210C213E2
:10038000C21C0800C201431308008518CC2919308B
:10039000C1070318D12908000A30C102031CE32950
:1003A0000800FF30C1004214643040020318080006
:1003B000421042154317C310F51BC3147717E617F5
:1003C0002A30C8000800C1014210C213421D0800B3
:1003D000C20143130800E303031D0800E0080319EA
:1003E000FE2965186008E51861086519620899001A
:1003F0000330E3000310E50DE51D08001430E300B1
:100400000130E500EE080319102AEE0303190E2A45
:100410006030E605031D102AE00108001F30E604E5
:100420000310E40D03186414640866050319102A08
:100430002E2B8C1E0800E7174A150717FA30FD000F
:100440001819CA146908E8006A08E9001A08EA00DD
:10045000E81F08006808C13C031D362A69086A05C0
:10046000C3046A096904C3053625A12A6808C23C89
:10047000031D422A69086A05C5046A096904C5059D
:100480003C25A12A6808C43C031D492A6908F700D5
:10049000A12A6808FC39E03C031D5A2A690868183B
:1004A0008038BB006A08E8188038BA00B125BE144D
:1004B0003E14A12A6808FC39F03C031D772A69081C
:1004C00068188038EC008B136C0803178D008316B6
:1004D0008C130C1483120C080313ED008B176C03A0
:1004E00044300319ED003230EE00E616A12A680808
:1004F000FC39803C031D862A690868188038CE00C4
:100500006A08E8188038CF00D815A12A6808FC3995
:10051000903C031D912A690868188038CE0058164F
:10052000A12A6808A03C031DA12A69086A1880381E
:10053000CD00C310EA18C31445126A194516D8161F
:10054000A12A08005919AF2AD3030F305305031D00
:100550000800D3080319B22A0716D30E0800591B46
:100560008523591307125911D91891295518500884
:10057000D5185108551952085705031DC22AFF30D6
:10058000D300C52A2230D300C52A0310D70C031884
:10059000CA2A08008030D7000310D50DD519D12AFA
:1005A00008000130D5000430D819D4000830581A9A
:1005B000D4000310D40D031854145408580503191B
:1005C000D12A7923D9140800EF0B08000330EF007B
:1005D000061E0F2B05160310F00D031CFD2A01301B
:1005E000F0000310F10D711EFD2A0130F100F00042
:1005F0004408F300C31BF317051271187308F118B0
:10060000720871197708F11D082B4B084A188038B9
:100610007005061203198516031D851208000616BB
:100620000800DA0A0319D9165916071E5912D91DDE
:100630002A2B591A2A2BB1155A08283CD91A03100B
:10064000DD0DDC0DDB0DDA01D912DE0B2A2B3116A4
:100650001930DE00D915591ED9110800E001E10159
:10066000E201E41F3A2B4F30E0004808E10049085E
:10067000E200E613641F432B4830E0004E08E1001F
:100680004F08E2006613E41E4C2B4730E0006C0874
:10069000E1006D08E200E612641E582B4130E000D4
:1006A000390884000008E1003D0884000008E200E9
:1006B000E41D602B4C30E0007708E1007808E20090
:1006C000641D682B4530E0004A08E1004B08E20059
:1006D000E41C702B4630E0004308E1004408E200CF
:1006E000641C782B5830E0005930E1005A30E200A9
:1006F0000800D001D101D201541C832BF730D00067
:100700004308D100AB2BD41C8A2BA130D000770832
:10071000D100AB2B541D912BA230D0004508D10045
:10072000AB2BD41D9B2BC130D0004E08D1004F08FD
:10073000D200D8110800541EA32BC230D0004E089E
:10074000D1005812AB2BD41E0800A730D0004D08A2
:10075000D100D812AB2B50085106D2000800311F2F
:10076000B42BFC0303193113451BBB2B071FBB2BF9
:10077000FD0303190713C70BDF2B8B1390300317EF
:100780008D0083168C130C1483120C080313C700FE
:100790008B170310B20D0F304418B200B21FD92BC3
:1007A000E6171E30C8003208C9004313321F4A162C
:1007B000B201431BCA11431B4A12CB1B4313071838
:1007C0004311071C43150719C311071DC3158719CA
:1007D0004312871D43168710751CF02BC31A87140C
:1007E000FE0B080044186426441C87127708780220
:1007F00003198716451F012C6026071F8716071B44
:1008000087124A1C87174A185C26790AF71BF707D4
:10081000771B0E2C790A77020318F7007808F2008C
:100820000310790C013E7802C3130318F200031879
:10083000C317C3120310790C013E46077802031850
:10084000C31646087802031CC3160310790C013E38
:100850004602031C08007802031CC3120800311171
:10086000311B0800591808004A100717FA30FD001C
:10087000B7010430B8000C30370230300318B80725
:10088000C319B8178B1320303707380703178D00AB
:1008900083168C130C1483120C080313A400A500F8
:1008A000C030A50610303707380703178D008316B0
:1008B0008C130C1483120C080313A300A60002303F
:1008C000A60600303707380703178D0083168C13F0
:1008D0000C1483120C080313A200A7000130A70612
:1008E0008B17B11F792C22090339A200A309A4098F
:1008F000A509C31D882C22082D02031D302D2308B5
:100900002E02031D302D24082F02031DE42C942CED
:1009100024082F02031D302D23082E02031DE42C72
:1009200022082D02031D302DE6170A30C8003708B3
:10093000C90000303702031DA22C431808004314DD
:100940003625080001303702031DB92CFF30FC00AA
:100950003117441CC314441C94257519B32C441836
:1009600043134418CA15441C43170130431BB200FB
:10097000080002303702031DCA2CFF30FC0031177B
:10098000441CC314441C9C25441C43170130431BC6
:10099000B200080003303702031DD12C441CC314DD
:1009A00008003030370738077F3903178D0083166A
:1009B0008C130C1483120C080313F7005917441CF2
:1009C0004225FF30FC003117C31DEB2C25082F02F8
:1009D000031D302DF32C26082E02031D302D270871
:1009E0002D02031D302DE6170C30C8003708C90052
:1009F00000303702031D012D431C0800431036252B
:100A0000080001303702031D182DFF30FC0031179C
:100A1000441CC310441C8B257519122D4418431314
:100A20004418CA15441C43170130431BB200080088
:100A300002303702031D292DFF30FC003117441C02
:100A4000C310441C9C25441C43170130431BB200B7
:100A5000080003303702031D302D441CC31008006A
:100A6000B70A1C30370203180800392C2130BB00AC
:100A70004308BA00B12508002330BB004508BA007E
:100A8000B1250800771B0800431A892D0310790C43
:100A9000013E77020318F7000318462D7708780205
:100AA0000319642D03185C2D78087702C3187902A6
:100AB000C318013EFF006B2D77087802C31C790232
:100AC000C31C013EFF006B2D0310790C013EFF009B
:100AD000F518F7077E2D0310790C013EF518013E3D
:100AE0007F02031C7E2D0310790C013EF707790A63
:100AF00077020318F7000318772D7E2D7708780208
:100B00004313031D4317F51843170130431BB2006D
:100B100008007E2D08005917C310780AF700790ADB
:100B200077020318F70008005917C3147803F70079
:100B3000790AF71BF707080059170310790C780793
:100B40007902031CAB2D0319AB2D0310790C013E68
:100B50007807F70008000310790C013E7802F700CF
:100B60000800FF010530DF000D123B088312031758
:100B70008D00831203133A08831203178C00831627
:100B800003178C130C158B138B1BC32D55308D0045
:100B9000AA308D008C148B170C1183120313640080
:100BA000DF03031DD82D0530DF00FF030319DB2D04
:100BB0000D1ECF2D08000C118B17B12D8B138B1B25
:100BC000DE2D313003178D0083168C130C14831225
:100BD0000C080313F4008B1774108B1332300317B7
:100BE0008D0083168C130C1483120C080313F5006C
:100BF0008B178B13333003178D0083168C130C1453
:100C000083120C080313F6008B173E18242E8B1347
:100C1000213003178D0083168C130C1483120C08DB
:100C20000313C3008B1743138B13233003178D005B
:100C300083168C130C1483120C080313C5008B1736
:100C4000C5124510C51045138B13203003178D00B6
:100C500083168C130C1483120C080313C6008B1715
:100C6000460A0319C6018B13303003178D00831613
:100C70008C130C1483120C08031307183030F9007E
:100C8000F9038B13803003178D0083168C130C141B
:100C900083120C080313B9008B178B1381300317D1
:100CA0008D0083168C130C1483120C080313BD00E3
:100CB0008B17BE103E1008000708803A8700080016
:100CC0000708403A870008000708203A8700080014
:100CD000FF006426FF0B692E08000708023A870010
:020CE00008000A
:084000000F00000004000400A1
:02400E00CC03E1
:1042000000004400FF00FF00400042004400460060
:104210004200430040004100460047004400450082
:10422000FF00FF00FF00FF00F200F600FA00FE00B2
:10423000F000F200F400F600F800FA00FC00FE00C6
:10424000FF00FF00FF000000E500E500E500E500DD
:10425000E900E900E900E900E900E900E900E90016
:104260001800000001000000FF00FF00FF00FF0039
:104270000000010002000300040005000600070022
:104280004300420041004000470046004500440012
:104290004400450046004700400041004200430002
:1042A000F000F200F400F600F800FA00FC00FE0056
:1042B000F000F200F400F600F800FA00FC00FE0046
:1042C000ED00ED00ED00ED00ED00ED00ED00ED0086
:1042D000F100F100F100F100F100F100F100F10056
:1042E000080009000A000B000C000D000E000F0072
:1042F0001000110012001300140015001600170022
:104300007A007B00FF00FF000000000000000000BA
:104310000300030003000300030003000300030085
:10432000AA00FF00FF00FF00C800C800C800C800C6
:10433000C800C800C800C800C800C800C800C8003D
:10434000FF00FF00FF00FF00C300F300CF00FF00ED
:104350000300C3003300F3000F00CF003F00FF0055
:10436000FF00FF00FF00FF00FF00FF00FF00FF0055
:10437000FF00FF00FF00FF00FF00FF00FF00FF0045
:10438000020002000200020002000200020002001D
:10439000000000000000000000000000000000001D
:1043A000C800C800C800C800C800C800C800C800CD
:1043B00088008800880088008800880088008800BD
:1043C0000300C3003300F3000F00CF003F00FF00E5
:1043D0000300C3003300F3000F00CF003F00FF00D5
:1043E000FF00FF00FF00FF00FF00FF00FF00FF00D5
:1043F000FF00FF00FF00FF00FF00FF00FF00FF00C5
:00000001FF
